:1000000080313E28080008007E14803120007F08DF
:10001000F6002100111C13282000111C13289D310B
:10002000A225803139282100911D1D282000911D15
:100030001D288E31BB26803139282100921D2728AA
:100040002000921D2728803102208031392821008C
:10005000911E31282000911E31289E31AD2680311D
:1000600039282100111E39282000111E39289E31FF
:100070008E2676082000FF007E100900803140287F
:10008000F701F801F901FA01FB0163308400003047
:1000900085000D309D319C2580312100E701E8016C
:1000A000E901EA01EB01EC015930840001308500DF
:1000B0000A309D319C258031DB3084000130850081
:1000C00008309D319C258031A030840002308500AD
:1000D00040309D319C258031CD3084009D3085009D
:1000E00063308600013087000A309D3196258031CB
:1000F000EB30840090308500A0308600013087000E
:100100003B309D3196258031003084009030850051
:10011000203086000230870024309D3196257E10E5
:1001200020009331302B0034C13481344034013409
:10013000C034803441340134C0348034413400341C
:10014000C134813440340134C0348034413400340B
:10015000C134813440340034C134813440340134FA
:10016000C034803441340134C034803441340034EC
:10017000C134813440340034C134813440340134DA
:10018000C034803441340034C134813440340134CB
:10019000C034803441340134C034803441340034BC
:1001A000C134813440340134C034803441340034AB
:1001B000C134813440340034C1348134403401349A
:1001C000C034803441340034C1348134403401348B
:1001D000C034803441340134C0348034413400347C
:1001E000C134813440340034C1348134403401346A
:1001F000C034803441340134C0348034413400345C
:10020000C134813440340134C0348034413400344A
:10021000C134813440340034C13481344034013439
:10022000C034803441340134C0348034413400342B
:10023000C134813440340034C13481344034013419
:10024000C034803441340034C1348134403401340A
:10025000C034803441340134C034803441340034FB
:10026000C134813440340034C134813440340134E9
:10027000C034803441340134C034803441340034DB
:10028000C134813440340134C034803441340034CA
:10029000C134813440340034C134813440340134B9
:1002A000C034803441340034C134813440340134AA
:1002B000C034803441340134C0348034413400349B
:1002C000C134813440340134C0348034413400348A
:1002D000C134813440340034C13481344034013479
:1002E000C034803441340134C0348034413400346B
:1002F000C134813440340034C13481344034013459
:10030000C034803441340034C13481344034013449
:10031000C034803441340134C0348034413400343A
:10032000C134813440340034C034C1340134C33466
:1003300003340234C234C63406340734C7340534B7
:10034000C534C4340434CC340C340D34CD340F34BF
:10035000CF34CE340E340A34CA34CB340B34C934DF
:1003600009340834C834D83418341934D9341B3417
:10037000DB34DA341A341E34DE34DF341F34DD3437
:100380001D341C34DC341434D434D5341534D7340F
:1003900017341634D634D23412341334D3341134DF
:1003A000D134D0341034F03430343134F134333487
:1003B000F334F23432343634F634F7343734F53437
:1003C00035343434F4343C34FC34FD343D34FF34BF
:1003D0003F343E34FE34FA343A343B34FB3439345F
:1003E000F934F83438342834E834E9342934EB3437
:1003F0002B342A34EA34EE342E342F34EF342D34B7
:10040000ED34EC342C34E43424342534E53427340E
:10041000E734E63426342234E234E3342334E1345E
:1004200021342034E034A03460346134A1346334A6
:10043000A334A23462346634A634A7346734A534B6
:1004400065346434A4346C34AC34AD346D34AF34BE
:100450006F346E34AE34AA346A346B34AB346934DE
:10046000A934A83468347834B834B9347934BB3416
:100470007B347A34BA34BE347E347F34BF347D3436
:10048000BD34BC347C34B43474347534B53477340E
:10049000B734B63476347234B234B3347334B134DE
:1004A00071347034B03450349034913451349334C6
:1004B0005334523492349634563457349734553436
:1004C0009534943454349C345C345D349D345F34BE
:1004D0009F349E345E345A349A349B345B3499345E
:1004E00059345834983488344834493489344B3436
:1004F0008B348A344A344E348E348F344F348D34B6
:100500004D344C348C34443484348534453487340D
:10051000473446348634823442344334833441345D
:10052000813480344034013400340A34003464347B
:100530000034E834033410342734453472347234D0
:100540006F3472343A3420344D34533450344C3494
:100550005F3452346534613464344D346234503421
:10056000643475343A3420344D34533450344C347C
:100570005F345234653461346434503461346334EC
:100580006B346534743420346634613469346C34CB
:1005900065346434203472346534613464346934CD
:1005A0006E34673420344634433430347834303455
:1005B00046342F34303478343134303420345034AD
:1005C0004434553400344534723472346F347234E8
:1005D0003A3420344D34533450344C345F34523434
:1005E0006534613464344D34623450346434753469
:1005F0003A3420344D34533450344C345F34523414
:100600006534613464345034613463346B3465343C
:10061000743420346634613469346C346534643441
:100620002034723465346134643469346E34673430
:100630002034623461346C3461346E346334653434
:1006400020346F346634203450344434553400340C
:100650005734613472346E3469346E3467343A34EA
:10066000203455346E3473347534703470346F34D0
:1006700072347434653464342034663475346E34C2
:100680006334743469346F346E34203463346F34BB
:10069000643465342C342034733465346E346434FB
:1006A00069346E34673420346534783463346534A7
:1006B0007034743469346F346E3420347234653479
:1006C000733470346F346E347334653400342A34C8
:1006D0002A342A342A3420344D346F34643462345A
:1006E00075347334203453346C3461347634653467
:1006F0002034503472346F3474346F3463346F3454
:100700006C3420344C346934623472346134723461
:1007100069346534733420342D34203443346F34D9
:100720006C34773461347934203453346F346C341E
:100730007534743469346F346E34733420342A342D
:100740002A342A342A3400342A342A342A342A34E3
:100750002A342A342A342A342A342A342A342A34A9
:100760002A342A34203468347434743470343A347B
:100770002F342F347734773477342E3463346F3416
:100780006C3477346134793473346F346C34753449
:10079000743469346F346E3473342E3463346F348C
:1007A0006D3420342A342A342A342A342A342A3420
:1007B0002A342A342A342A342A342A342A342A3449
:1007C00000344534723472346F3472343A34203425
:1007D0004D34533450344C345F34523465346134C6
:1007E00064344D3462345034643475343A342034D3
:1007F0004D34533450344C345F34523465346134A6
:1008000064345034613463346B346534743420346C
:100810006634613469346C34653464342034723441
:1008200065346134643469346E346734203446345A
:10083000433400344534723472346F3472343A3491
:1008400020344D34533450344C345F345234753486
:100850006E344D346F3464346234753473343A34E6
:1008600020344534723472346F347234203472342C
:1008700065346134643469346E346734203441340F
:10088000643464346934743469346F346E3461347C
:100890006C342034413464346434723465347334D9
:1008A000733400343C343D343D34203442347234AB
:1008B0006F34613464346334613473347434203499
:1008C0006D346534733473346134673465342C3477
:1008D00020346E346F3420347234653473347034A1
:1008E0006F346E347334653420347434723461344C
:1008F0006E3473346D3469347434743465346434F0
:100900002E3400343C343D343D342034533475347B
:1009100063346334653473347334663475346C34DF
:100920006C34793420347434723461346E347334FA
:100930006D3469347434743465346434203445342B
:100940007834633465347034743469346F346E349D
:10095000203472346534733470346F346E347334CD
:10096000653400343C343D343D34203453347534E4
:1009700063346334653473347334663475346C347F
:100980006C34793420347434723461346E3473349A
:100990006D346934743474346534643420344E34C2
:1009A0006F3472346D3461346C3420347234653495
:1009B000733470346F346E347334653400344D34B2
:1009C000533450344C345F3449346E3469347434A5
:1009D0007C34203449346E3469347434693461347D
:1009E0006C34693473346534643420346C34693461
:1009F000623472346134723479342034733475342F
:100A000063346334653473347334663475346C34EE
:100A10006C34793400344534723472346F34723447
:100A20003A3420344D34533450344C345F345234DF
:100A300075346E344D346F346434623475347334C9
:100A40003A3420344534723472346F347234203482
:100A5000723465346134643469346E3467342034FC
:100A600043345234433400344534723472346F3476
:100A700072343A3420344D34533450344C345F346F
:100A8000523475346E344D346F346434623475349A
:100A900073343A34203457347234693474346534DE
:100AA00050346F34723474342034663461346934B1
:100AB0006C346534643400343D343D343E34203489
:100AC000463443343D343034783431343034203497
:100AD00028345734723469347434653420344D34D6
:100AE00075346C347434693470346C346534203447
:100AF0005234653467346934733474346534723411
:100B00007334293400343D343D343E34203446348B
:100B100043343D3430347834303433342034283462
:100B20005234653461346434203448346F346C3466
:100B3000643469346E346734203452346534673435
:100B40006934733474346534723473342934003442
:100B50003D343D343E342034463443343D34303427
:100B6000783430343634203428345734723469348D
:100B7000743465342034533469346E3467346C34DF
:100B800065342034523465346734693473347434D2
:100B900065347234293400343D343D343E342034DD
:100BA000463443343D3430347834303446342034A1
:100BB00028345734723469347434653420344D34F5
:100BC00075346C347434693470346C346534203466
:100BD00043346F3469346C347334293400343D3415
:100BE0003D343E342034463443343D34303478345C
:100BF000303434342034283452346534613464342D
:100C0000203449346E3470347534743420345234A2
:100C100065346734693473347434653472347334CE
:100C2000293400343D343D343E342034463443349A
:100C30003D3430347834303435342034283457342B
:100C400072346934743465342034533469346E3406
:100C500067346C346534203443346F3469346C3415
:100C60002934003442347534663466346534723461
:100C7000203474346F346F34203473346D34613401
:100C80006C346C34203474346F34203472346534F2
:100C9000613464342034503444345534003457348F
:100CA000613472346E3469346E3467343A342034CB
:100CB00053346C34613476346534203449344434EC
:100CC00020346D34693473346D3461347434633476
:100CD000683400343D343D343E34203446344334AB
:100CE0003D34303478343034313420342834523484
:100CF000653461346434203443346F3469346C3483
:100D00007334293400343D343D343E342034463489
:100D100043343D3430347834303432342034283461
:100D200052346534613464342034443449342934D1
:100D300000344534723472346F3472343A342034AF
:100D400043345234433420346D34693473346D3455
:100D5000613474346334683400344E346534773429
:100D600020344D346F346434623475347334203439
:100D700052346534713475346534733474340034EA
:100D80006D347334673431340034253464340034C2
:100D90002000E000DF01A0019830A1008630A20011
:100DA000600880310320863120302000B6000130F9
:100DB000B7000130B8000030B90060089F31D42777
:100DC00086312000D8005808DF005F080319F22E92
:100DD000A001A00A1A30A1008430A200600880316E
:100DE0000320080020006008D8005808A000220056
:100DF00020089D31B1258631013A0319032F2200C5
:100E00002008031DCF2F20302000D8005808C00034
:100E100060088831342086312000D9005908DF006D
:100E20005F080319172F0A305F06031D08005F08CB
:100E3000031D522F22005808013E203E2000B6001C
:100E4000B7010130B73D0230B8000030B90060088A
:100E50009F31D42786312000D8005808DF005F0872
:100E600003193D2FA001A00A0B30A1008530A2007C
:100E70006008803103208631522F20302000D800B6
:100E80005808A30060089331F5238631013A03190D
:100E9000522F07302000D8005808DF0060089D312D
:100EA0008A25863120005F0803195A2F0A305F0611
:100EB000031D08005F08031D692F0430D80058087F
:100EC000A000AD30A1008630A20060088031032070
:100ED000863120302000D8005808D100A030D90039
:100EE0005908D20060089531F32586312200200888
:100EF0000319C22F21005808033E2000DB000030F8
:100F000003180130DC005C08A3005B08A2005D3020
:100F1000D8005808A400A030D9005908A5005F30B7
:100F2000DA005A08A6006008903151208631003A54
:100F3000031DA52F2000A001A00A3430A100853098
:100F4000A20060088031032008002100A11FB52FF6
:100F500003302000D8005808A0008230A10084305F
:100F6000A200600880310320080003302000D80070
:100F70005808A000B230A1008430A200600880317F
:100F80000320080004302000D8005808A000523088
:100F9000A1008430A20060088031032008000630E0
:100FA0002000D8005808DF000230D8005808A00000
:100FB0004F30A1008630A2006008803103208631C6
:100FC000200060089D318A250800E9302000A0003B
:100FD0002008E400E930A0002008E300E5146510D3
:100FE000E7018030240094002830950097010930F3
:100FF0009200200091112100911508000130080095
:101000002000A700A901AA01A8012208A400210824
:10101000A300A335A40D2808A500A60124082602D4
:10102000031D142823082502031808002908270790
:10103000A30023088600013087000108A4002A08C5
:101040002007A500250886008701240881000130BB
:10105000A3002308A9070130A3002308AA07013031
:10106000A3002308A80705282000C800C7014008DE
:10107000013EB6000130B7000130B8000030B900C1
:1010800048089F31D42788312000C1004108C7009B
:10109000470803199728A001A00AE130A100833076
:1010A000A2004808803103208831FF280430200046
:1010B000C5000030C60002307E284008023EB6005F
:1010C0000130B7000530B8000030B90048089F3142
:1010D000D42788312000C1004108C7004708031DFC
:1010E00082284008063E8600013087000108C100C2
:1010F000C2014108C5004208C6000730C3000030E5
:10110000C400B628A001A00A9D30A1008230A20030
:101110004808803103208831B6280A302000C100F9
:101120004108C70048089D318A258831B62820002B
:10113000400A8600013087000108013A0319562849
:10114000033A03195628013A03195628073A031996
:101150005628013A03195628033A03195628093A22
:1011600003195D281F3A03195D288D2820004708C0
:10117000031DFF2800304602393003194502031CC5
:10118000D5280830C1004108C700A001A00A3230AC
:10119000A1008630A2004808803103208831200059
:1011A00048089D318A258831FF28200040084307E0
:1011B000B6000130B7004608B9004508B800480835
:1011C0009F31D42788312000C1004108C70047085B
:1011D0000319F328A001A00AE330A1008230A20085
:1011E000480880310320200043084507FF3EC10026
:1011F0004008383E86000130870041088100200009
:10120000470808002000BB003030B2003208B600AA
:101210002F08B3002E08B200AE0A0319AF0A320835
:101220008400330885000008B4003408BC003C0882
:101230000319CB2925303C0603192A293C08B200A2
:101240003B0886008701320881000130B200320875
:10125000BB070829B7012F08B3002E08B200AE0A59
:101260000319AF0A32088400330885000008BC0067
:10127000003A0319CB29643A031942290D3A03199C
:1012800042290829360886008701403FB900413FBE
:10129000BA000230B2003208B607BA1F582903302C
:1012A000B2003208B704B909BA09B90A0319BA0A6F
:1012B000BC01BC0A05303C0603197D293C08B2007C
:1012C000B301B235B30D9330320784008230333D21
:1012D0008500003FB400013FB50035083A02031D08
:1012E000732934083902031C7D290130B200320809
:1012F000BC0705303C06031D5E2937080339031976
:101300008C292D30B2003B0886008701320881000D
:101310000130B2003208BB073C08B2003208B80006
:10132000FF30B2003208B807380A031908290A301A
:10133000A8000030A9003808B200B301B235B30DDF
:101340009330320784008230333D8500003FA00097
:10135000013FA1003A08A3003908A2009031802083
:10136000893120002108AB002008AA0090312420F8
:10137000893120002808303EB4003408BC003C0805
:10138000B2003B0886008701320881000130B200BC
:101390003208BB0790293B088600870181010800BD
:1013A0002000C5003D08023E86000130870001088C
:1013B000BF00C0013F08C000BF013F08C200400895
:1013C000C3003D08033E8600013087000108BF00CE
:1013D000C0013F08C2044008C3043D08043E860023
:1013E000013087000108BF00C0013F08C000BF01F5
:1013F0003F08C6004008C7003D08053E8600013092
:1014000087000108BF00C0013F08C6044008C704A8
:101410003D0A86000130870003300106031D182AAB
:101420000330BF003F08A0008330A1008530202A90
:1014300003302000BF003F08A000EF30A10085303E
:10144000A200450880310320893120004608470466
:1014500003199D2A003047027E3003194602031803
:101460009D2A4508BF003F08A0003D0886000130C6
:1014700087000130413FA1004308A3004208A200B9
:101480004708A5004608A4003D08860001308700F3
:101490000108963190268931013A031D9A2A2000CD
:1014A0004508BF003F08B0003D08860001308700B6
:1014B0000130413FB1004308B3004208B200470881
:1014C000B5004608B4003E08033EC0004008B60020
:1014D0003D0886000130870001088A31A322893146
:1014E0002000C1004108C4004408031D982A3D0A99
:1014F0008600013087000108BF003E0A8600870190
:101500003F0881004635BF003E08023E8600870145
:101510003F0881003E08023E860087010108023E26
:10152000BF003E08383E860087013F088100A12A9F
:1015300004309E2A023020009E2A0330BF003F085C
:10154000C40044080800742B20003208B43EA000F8
:101550000130A1003608B7003708A2003508A40002
:101560003408A3009231D0228A31832B2000320824
:10157000343EA0000230A1003608B7003708A200B0
:101580003508A4003408A3009231D0228A31832B7D
:101590000030200033020A30031932020318E12A16
:1015A0003235A03EA0000130A1003608B700370850
:1015B000A2003508A4003408A300913126218A3105
:1015C000832B003020003302143003193202031C35
:1015D000182B003033021E30031932020318182B67
:1015E0000330B7003708A0003208EC3EB800FF30E7
:1015F000333DB900B936B80C38089E310A268A3115
:10160000C43E2000BA003A08BC003608B7003708CC
:10161000A4003508B9003408B800B936B80C380849
:10162000A5003908A6003C08933190238A31832B0A
:10163000003020003302283003193202031C442BEF
:10164000003033023230031932020318442B3608BB
:10165000B7003708A0003508B9003408B800B9361B
:10166000B80C3808A1003908A2003208D83EBA00E8
:10167000FF30333DBB00BB36BA0C3A080907633E66
:10168000923173228A31832B0030200033023C30A8
:1016900003193202031C832B00303302403003193C
:1016A00032020318832B3608B7003708A00035082C
:1016B000A2003408A1003235883ED33E8831002094
:1016C0008A31832B20003235203EA0000230A10059
:1016D0003608B7003708A2003508A4003408A30074
:1016E000913126218A31832B20003108013A0319D8
:1016F000A42A033A0319B62A013A0319C82A073A59
:101700000319622B832B003008002000C5003D0820
:10171000023E8600013087000108BF00C0013F087B
:10172000C000BF013F08C2004008C3003D08033E9F
:101730008600013087000108BF00C0013F08C204D5
:101740004008C3043D08043E8600013087000108BC
:10175000BF00C0013F08C000BF013F08C6004008ED
:10176000C7003D08053E8600013087000108BF0024
:10177000C0013F08C6044008C7043D0A8600013086
:1017800087000103031DCC2B0330BF003F08A000DE
:101790006A30A1008630D42B03302000BF003F0800
:1017A000A0008330A1008630A200450880310320CC
:1017B0008B3120004608470403196D2C0030470286
:1017C00081300319460203186D2C4508BF003F08FD
:1017D000A0003D088600013087000130413FA10094
:1017E0004308A3004208A2004708A5004608A40039
:1017F0003D088600013087000108963190268B3124
:10180000013A031D6A2C20004508BF003F08B000C4
:101810003D088600013087000130413FB100430898
:10182000B3004208B2004708B5004608B4003E08BD
:10183000033EC0004008B6003D0886000130870026
:1018400001088A31A3228B312000C1004108C40065
:101850004408031D682C3D0A8600013087000108FA
:10186000BF003E0A860087013F0881004708C0008C
:101870004608BF00C036BF0CC036BF0CC036BF0C18
:101880003F08C1003E08023E8600870141088100F2
:1018900007304605BF0000304705C0003F08400440
:1018A00003195A2C0130BF003E08023E8600870112
:1018B0003F0881073E08023E860087010108023E7C
:1018C000BF003E08383E860087013F088100712C2A
:1018D00004306E2C023020006E2C0330BF003F0815
:1018E000C400440808002000C900CB010430C30034
:1018F0004308C6000130CC000030CD004108023E54
:101900008600013087000108C300C4014308C400F9
:10191000C3014308C7004408C8004108033E8600CD
:10192000013087000108C300C4014308C70444080C
:10193000C804410A86000130870010300106031DEB
:10194000E02C4108043E8600013087000108C300F6
:10195000C4014308C400C3014308CC004408CD00BF
:101960004108053E8600013087000108C300C4011C
:101970004308CC044408CD044C084D040319D72C6B
:1019800000304D027C3003194C020318D72C4D084F
:10199000C4004C08C300C335C40D4108063E860090
:1019A000013087000108430644040319DC2C03308E
:1019B000C3004308CB00E02C0730C3004308C60037
:1019C000410A86000130870006300106031DF02C15
:1019D0000330C3004308A000A830A1008530F82CD4
:1019E00003302000C3004308A0005C30A100853014
:1019F000A2004908803103208C3120004B08031DD0
:101A0000762D4908C3004308A00041088600013034
:101A100087000130413FA1004808A3004708A20009
:101A20004D08A5004C08A40041088600013087003D
:101A30000108963190268C31013A031D712D20004A
:101A40004908C3004308B3004108860001308700FD
:101A50000130413FB4004808B6004708B5004D08C2
:101A6000B8004C08B70041084607B9000130BA0079
:101A700041088600013087000108973139278C31F1
:101A80002000C4004408CB004B08031D6F2DCA0181
:101A9000CA0A06304A020318662D4A084107C300E5
:101AA00043088600013087000108C4004A08420745
:101AB000C500450886008701440881000130C30045
:101AC0004308CA0706304A02031C4D2D0530C300E7
:101AD0004208383E8600870143088100762D043095
:101AE000732D02302000C3004308CB004B080800D0
:101AF0002000CB00CE010130CF000030D0004108E3
:101B0000023E8600013087000108C300C40143087B
:101B1000C400C3014308C9004408CA004108033E89
:101B20008600013087000108C300C4014308C904CE
:101B30004408CA04410A8600013087000F300106BC
:101B4000031DF72D4108043E86000130870001087F
:101B5000C300C4014308C400C3014308CF004408C4
:101B6000D0004108053E8600013087000108C3000F
:101B7000C4014308CF044408D0044F08500403199B
:101B8000ED2D00305002813003194F020318ED2D66
:101B90005008C4004F08C300C436C30CC436C30C7D
:101BA000C436C30C4308C5004508C80007304F05BC
:101BB000C30000305005C400430844040319E42D59
:101BC0000130C3004308C8074108063E86000130C3
:101BD0008700010848060319F22D0330C3004308AB
:101BE000CE00242E4108073EC6000130232E4108B6
:101BF000043E8600013087000108031D092E4108BC
:101C0000053E8600013087000108031D092ECC0126
:101C1000202E4108043E860001308700010A031D82
:101C20001C2E4108053E8600013087000108031D77
:101C30001C2ECC01CC0A202E0330C3004308CE005A
:101C40004C30C6000030C700410A860001308700D2
:101C500005300106031D342E0330C3004308A000E5
:101C60001230A10086303C2E03302000C300430810
:101C7000A000CC30A1008530A2004B0880310320A9
:101C80008D3120004E08031DB92E4B08C3004308B8
:101C9000A00041088600013087000130413FA100CB
:101CA0004A08A3004908A2005008A5004F08A40054
:101CB00041088600013087000108963190268D3159
:101CC000013A031DB42E20004B08C3004308B300A3
:101CD00041088600013087000130413FB4004A08C6
:101CE000B6004908B5005008B8004F08B7004708CB
:101CF000BA004608B9004108860001308700010893
:101D0000973139278D312000C4004408CE004E0899
:101D1000031DB22ECD01CD0A06304D020318A92EA7
:101D20004D084107C30043088600013087000108C1
:101D3000C4004D084207C5004508860087014408D5
:101D400081000130C3004308CD0706304D02031C5B
:101D5000902E0530C3004208383E860087014308B4
:101D60008100B92E0430B62E02302000C300430893
:101D7000CE004E080800200091112400951FF42F7A
:101D800095132000EE017808023E860087010108C5
:101D9000860087018101810AF8010800E518080022
:101DA0006408F2007208F8006408860087010108E0
:101DB000F2007208EF00640886008701413FF900D5
:101DC0000430F2007208E4076408ED3A031DEC2EBB
:101DD000E930F2007208E400651064086306031934
:101DE000E514240016140230F20072082000EE0000
:101DF0000800240096140230F20072082000EE0061
:101E000008002400161F0D2F0130F2007208200078
:101E1000E70704309E31402608007B08F3007A086B
:101E2000F200F336F20C7208240091007A1C1E2F87
:101E30000B30F20072082000EE0008000330F200C0
:101E400072082000EE0008002400161F302F013019
:101E5000F20072082000E70704309E314026080097
:101E600096147B08F3007A08F2007308F200F3017D
:101E700006307205F40000307305F500F03074048C
:101E8000FA0000307504FB007A142000E801E80A2B
:101E90000230F2007208EE00080068030319662F92
:101EA0007908860001308700403FFA00413FFB007F
:101EB00079088600013087000130433FEA00790845
:101EC0008600013087000130423FE9007A08240093
:101ED00091007A1C712F0530F20072082000EE008C
:101EE00008000330F20072082000EE000800240011
:101EF000161F852F0130F20072082000E70724002A
:101F0000161305309E314026080001302000E902FA
:101F1000690A031D9F2F0530F2007208F90701308E
:101F2000EF02031D972F00309E3140260800240049
:101F300096140230F20072082000EE0008006A08D1
:101F4000860087010108240091000130F200720828
:101F50002000EA0708002400161FB92F0130F20004
:101F600072082000E70704309E3140262400161333
:101F7000080096150830F20072082000EE000800F4
:101F80000830F2007208EE002400961508002400C4
:101F90001108F20020006A0886008701720881009B
:101FA0000130F2007208EA070130E9020319E02F5C
:101FB000240096120630F20072082000EE00E42F92
:101FC000240096169D31E7252400161608000030DF
:101FD0009E31402608000130F20072082000E70719
:101FE00006309E314026080020006E0884000C3028
:101FF00004020318EB2F98310435003E82000800DC
:1020000002342234043444340634663408348834C8
:102010000A34AA34013411340334333405345534CA
:1020200007347734093499340134013400340034EE
:1020300001340134013401340034003400340034FC
:102040000134003401340034200028082904031925
:102050004C28AD01AD0AA91B37280130A835A90DC0
:10206000890B2E280130AC002C08AD072B2829083D
:102070002B02031D3D2828082A02031C4328280898
:10208000AA022908AB3B0130A936A80C890B4428C9
:102090000130AD02031D37282B08A9002A08A8002B
:1020A00008002000A801A80AEB012100E701F701C0
:1020B0002000A901AA0123082A02031D6128220881
:1020C00029020318732829082507A7002708860076
:1020D000870101089F315B27903101302000A9075B
:1020E0000030AA3D5B282408860087012208C03FF3
:1020F0002308C13F260886008701810128080800BF
:102100002000A501A601200821040319B028A70179
:10211000A70AA11B95280130A035A10D890B8C2899
:102120000130A4002408A70789280130A535A60D91
:10213000890B962821082302031DA02820082202CB
:10214000031CA7282008A2022108A33B2514013064
:10215000A136A00C890BA8280130A702031D9528E1
:102160002608A1002508A00008002000AA01AB0154
:10217000A9012408A6002308A500A535A60D290855
:10218000A700A80126082802031DC8282508270241
:10219000031808002A08A500A601250820078600C4
:1021A0002608213D87000108A7002B082207A80068
:1021B0002808860001308700270881000130A5002B
:1021C0002508AA070130A5002508AB070130A500A6
:1021D0002508A907B9280134113402342234033404
:1021E0003334043444340534553406346634073407
:1021F000773408348834093499340A34AA340034E2
:10220000003401340134003400340034003401342B
:1022100001340134013400340134003400347134A9
:10222000453441341F346334423478348B3443347E
:102230004F3475344434E1340334423443344F343E
:102240004C34573441345934003400342000AC014C
:10225000AD01AB012B08A500A60124082602031D31
:10226000332923082502031808002C08A500A6011D
:10227000A535A60D2508200786002608213D8700E4
:10228000403FA700413FA8002808A9002D082207C9
:10229000AA002A0886008701290881000130A500CC
:1022A0002508AD072C08A500A601A535A60D250813
:1022B000200786002608213D87000108A7002D0879
:1022C0002207A8002808860087012708810001301E
:1022D000A5002508AD070130A5002508AC07013091
:1022E000A5002508AB072A292000AC01AD01AB01F0
:1022F0002B08A500A60124082602031D8129230816
:102300002502031808002C08A500A60125082007AF
:1023100086002608213D87000108A700A80127089C
:10232000A800A7012D352207AA002A08860001303F
:1023300087002708C03F2808C13F2C08013EA500A0
:10234000003003180130A600250820078600260863
:10235000213D87000108A700A8012D352207A9000B
:1023600029088600013087002708810441312808A8
:1023700081040130A5002508AD070230A50025081D
:10238000AC070130A5002508AB0778292000AA0179
:10239000AB01AD012D08A500A60124082602031DEE
:1023A000D3292308250203180800AC01AC0AAE01AA
:1023B00008302E020318152A2A08A500A6012508B0
:1023C000200786002608213D870001082C05A7006C
:1023D0002E0AEB29A736890BEA292708A8002B0823
:1023E0002207A900290886000130870028088100FB
:1023F0000130A5002508AB070310AC0D0130A50086
:102400002508AD072D08A500A60124082602031DF6
:102410000B2A23082502031808000130A50025080F
:10242000AE0708302E02031CDC290130A500250868
:10243000AA07CA29FF302000A1002108A600FF300A
:10244000A1002108A7002008383E86008701010866
:10245000013EA1002108A900A801290828020318AB
:102460005D2A28082007A1002108860087010108AD
:102470002706A200A3012208A4002308A50025081E
:10248000850024088400933084078030853D00084F
:102490002606A1002108A70025088500240884003D
:1024A000933084078130853D0008A1002108A600F3
:1024B0000130A1002108A8072D2A2708A10029081A
:1024C0002007A20022088600870121088100260833
:1024D000A1002908013E2007A200220886008701EA
:1024E0002108810008002000A900AA01AB01A80171
:1024F0002808A300A40122082402031D812A210820
:102500002302031808002A352907A30023088600A0
:1025100001308700403FA400413FA5002508A600E8
:102520002B082007A70027088600870126088100BE
:102530000130A3002308AB072A352907A30023088D
:102540008600013087000108A4002B082007A500A1
:10255000250886008701240881000130A300230894
:10256000AB072B082007A300230886008701810101
:102570000130A3002308AB072B082007A300230882
:102580008600870181010130A3002308AB070130D9
:10259000A3002308AA070130A3002308A807782A6C
:1025A0002000A901AA012408A6002308A500A63638
:1025B000A50CA636A50CA636A50C2508A70027084D
:1025C000A80007302305A50000302405A600250833
:1025D00026040319EF2A0130A5002508A807AB013E
:1025E00028082B02031808002B082207A50025083D
:1025F000860087018101AC0108302C0203182B2BC7
:102600002908200786002A08213D87000108A50027
:102610002C0A0B2BA535890B0A2B2508A6002B08A5
:102620002207A700270886008701260881040130B9
:10263000A9070030AA3D24082A02031D212B2308E4
:102640002902031808000130A5002508AC0708304E
:102650002C02031C002B0130A5002508AB07F02A33
:102660002100E301E4019E312E2693319E31702634
:1026700093318B170B172000181428001715C03042
:102680002000A7008630A8009F31362793319F3164
:10269000AA279331013A031D8E2B9D31A925933131
:1026A0002000E100E20161082100E300200062084F
:1026B0002100E4009D31C325933120002108210031
:1026C000E600200020082100E500C5302000AE0013
:1026D0008630AF00210066082000B10021006508A7
:1026E0002000B000D930893102219331D930200047
:1026F000A7000030A8009F31362793312000A701A2
:10270000A70A00309E31CE26933100308631C8268C
:10271000933121001110200011104D2B80313E28E3
:102720002000AA00AC01AF01AB012B08A700A80153
:1027300026082802031D9E2B2508270203180800DF
:102740002D308600870103302000A7002708A00055
:102750002C089E310A26933120002A07A800280859
:102760008400013085000430A90012001E00A90B6E
:10277000B52B20002E08A7002F082407A800280842
:1027800086008701270881000130A7002708AF07CE
:102790002D08A7002F082407A80028088600870115
:1027A000270881000130A7002708AF072F0824075A
:1027B000A70027088600870181010130A7002708AC
:1027C000AF072F082407A70027088600870181018B
:1027D0000130A7002708AF070130A7002708AC0782
:1027E0000130A7002708AB07952B2000A700FF307A
:1027F000A4002408AA00FF30A4002408AB0023088A
:10280000383E8600013087000108013EA4002408FC
:10281000AD00AC012D082C0203183B2C2C0823071B
:10282000A400240886000130870001082B06A500BB
:10283000A6012508A8002608A9002908850028085F
:102840008400933084078030853D00082A06A40068
:102850002408AB00290885002808840093308407E9
:102860008130853D0008A4002408AA000130A4009E
:102870002408AC070A2C2D082307A400240886008E
:102880000130870001082B06031D542C2D08013E42
:102890002307A400240886000130870001082A06C7
:1028A000031D542C01300800A001A00A9930A1009A
:1028B0008630A20027088031032000300800200065
:1028C000B101B10AB401B501B201B301AF01B00168
:1028D0002B08860087018101B201B3010030330269
:1028E0001430031932020318C42C9E311C26943173
:1028F00020002108B0002008AF006B0803197D2CD0
:10290000210091126708DB3E860001308700010834
:102910002000AC0034082907AD0035082A3DAE0080
:102920002D0886002E0887002C0881000130EB025C
:102930002100911601302000AC002C082100E7078F
:10294000383067020318E70101302000B407003077
:10295000B53D9E311C26943120002108B00020088E
:10296000AF0027083506031DB72C260834060319C7
:10297000C42C0130B2070030B33D003033021430B4
:1029800003193202031C752C27083506031DCA2CB7
:1029900026083406031DD82C280886008701340831
:1029A000C03F3508C13F2B08860087018101E02C1C
:1029B0000530AC002B08860087012C088100B1018E
:1029C000310808002000B201AF01AE012E08A900B5
:1029D000AA0128082A02031DEF2C27082902031840
:1029E0000800B001B1013208A900AA012908240792
:1029F00086002A08253D87000108AB00AC012B08A2
:102A0000AC00AB012B08B0002C08B1000130A900CC
:102A10002908B2073208A900AA012908240786005C
:102A20002A08253D87000108AB00AC012B08B00443
:102A30002C08B1040130A9002908B2073208A90006
:102A4000AA012908240786002A08253D87000108D5
:102A5000AB00AC012B08B0042C08B1040130A90074
:102A60002908B2073208A900AA012908240786000C
:102A70002A08253D87000108AB00AC012B08B004F3
:102A80002C08B1040130A9002908B2070330A900BD
:102A90002908A0002F089E310A269431200026071D
:102AA000AA002A08860001308700303084008501A2
:102AB00004302000AB0012001E00AB0B5B2D013078
:102AC0002000A9002908AF070130A9002908AE0796
:102AD000E62C2000AD01AC01AB012B08A500A6013E
:102AE00024082602031D762D23082502031808005A
:102AF0002D08A500A6012508200786002608213DEF
:102B000087000108A700A8012708A800A7012C3505
:102B10002207AA002A088600013087002708C03F44
:102B20002808C13F0130A5002508AD072D08A500E4
:102B3000A6012508200786002608213D87000108F8
:102B4000A700A8012C352207A9002908860001301A
:102B50008700270881044131280881040130A5003D
:102B60002508AD072D08A500A60125082007860029
:102B70002608213D87000108A700A8012C3522075F
:102B8000A900290886000130870027088104413107
:102B9000280881040130A5002508AD072D08A500EF
:102BA000A6012508200786002608213D8700010888
:102BB000A700A8012C352207A900290886000130AA
:102BC0008700270881044131280881040130A500CD
:102BD0002508AD070130A5002508AC070130A50088
:102BE0002508AB076D2D2000D700D6013E2E5108D9
:102BF000D3005308BD005208D4005408BE00570843
:102C00008B31852395312A2E5108D3005308BD00FE
:102C10005208D4005408BE0057088931D02195319C
:102C20002A2E5108D3005308C1005208D40054087A
:102C3000C20057088D31782595312A2E5108D300CE
:102C40005308C1005208D4005408C20057088C3100
:102C5000732495312000D5005508D6005D2ED6018D
:102C6000D60A0230D3005308A0002830A1008330D8
:102C7000A20057088031032095315D2E2000510AB3
:102C80008600013087000108013A0319F72D033A45
:102C90000319F72D013A0319042E073A0319042EDC
:102CA000013A0319112E033A03191E2E093A03198A
:102CB000112E1F3A03191E2E2F2E2000560803191D
:102CC0007D2E510A86000130870001088038D3002C
:102CD000520A86008701530881005608D300520823
:102CE000023E86008701530881000230D30052085B
:102CF000383E860087015308810051088600013064
:102D000087000108D300520886008701530881001C
:102D10005208D3005308A000570892311A22080025
:102D20001C2F2000952E9F2EA62E24082207A600D9
:102D30002508233DA700003027021130AF2E0030B8
:102D400023020A30031922020318B22E2408220794
:102D5000A6002508233DA700003027020B300319E9
:102D60002602152F00302302143003192202031CFF
:102D7000D02E003023021E30031922020318D02E59
:102D800024082207A6002508233DA7002608EC3EBC
:102D9000A800FF30273DA900003029020830ED2EA1
:102DA00000302302283003192202031CF02E0030C9
:102DB00023023230031922020318F02E24082207BE
:102DC000A6002508233DA7002608D83EA800FF300E
:102DD000273DA90000302902063003192802152FCB
:102DE000003023023C3003192202031C1A2F00304A
:102DF000230240300319220203181A2F2508A700C6
:102E00002408A600A635A70D22082607A800230837
:102E1000273DA9002808C43EAA00FF30293DAB0089
:102E200000302B02093003192A0203181A2FAC01B3
:102E3000AC0A372FAC01372F20002108013A0319C3
:102E4000912E033A0319922E013A0319932E073A51
:102E50000319942E013A0319952E033A03199F2E54
:102E6000093A0319952E1F3A03199F2E1A2F2C0881
:102E70000800EF2F20003A08A1003908A00035080B
:102E8000B43EBB003B08A2003808A4003708A300EA
:102E90009131C6219731FE2F0030200036020A30D2
:102EA000031935020318652F3A08A1003908A0005C
:102EB0003535A03EBB003B08A2003808A400370807
:102EC000A300913174219731FE2F0030200036028B
:102ED000143003193502031C9F2F003036021E30B8
:102EE0000319350203189F2F0330BB003B08A000D5
:102EF0003508EC3EBC00FF30363DBD00BD36BC0C95
:102F00003C089E310A269731C43E2000BE003E0890
:102F1000C0003A08A5003908A4004008BB003B08DF
:102F2000A6003808BD003708BC00BD36BC0C3C0804
:102F3000A7003D08A8009431E2249731FE2F00300D
:102F400020003602283003193502031CCE2F003032
:102F500036023230031935020318CE2F3A08A10089
:102F60003908A0003508D83EBB00FF30363DBC0014
:102F7000BC36BB0C3B080907633EBD003D08A20000
:102F80003808BF003708BE00BF36BE0C3E08A3009D
:102F90003F08A400953169259731FE2F00302000AD
:102FA00036023C3003193502031CFE2F0030360276
:102FB0004030031935020318FE2F3A08A1003908E2
:102FC000A0003535883ED33EBB003B08A200380840
:102FD000A4003708A3009031B5209731FE2F2000C0
:102FE0003408053A03193A2F033A03194C2F093ACA
:102FF00003193A2F1F3A03194C2FFE2F00300800F7
:103000008E31CE2E8E31F92E8F314D2F8F31772F7D
:103010008F31E72F8F31AB2F8F31C02F8F31E72FBB
:103020008F31C72F8F31EB2F8F31012F8F31242F0D
:103B14002000EB012100E701F70108006A302100D1
:103B240099009A0198010800FE0012001E00FE0B85
:103B3400972D0034640080010131890B9D2D0034E0
:103B4400200011107D0897007C08960008002800CA
:103B540015082000A0002008A1002108080020006A
:103B6400A1002103031DB82D013008000030080016
:103B74000530280097000530960095012000931029
:103B8400080020001708A3001608A2002308A100BB
:103B94002208A00008004E346134813470341D348E
:103BA400C834D33467346634FF3489302000980035
:103BB400103099008030970096011708FD00160810
:103BC400FC0011102100111408000530F0007008E9
:103BD400F90701302000EF02031DF52D0430F00039
:103BE4007008EE000800EE01EE0A08002000A300B1
:103BF4002308A1000430A136890BFD2D2108A20061
:103C04002208A30023080F39A1002108A3000800FB
:103C14002000A300A201231C132E2008A1002108C8
:103C2400A2070310A00D0310A30C2308031D0D2EDF
:103C3400220808002100911220006B08A200A301B1
:103C44002208A4002308A5002100911620002508BD
:103C5400A1002408A00008009D3190259E319F31C9
:103C640013279E319D31BA259E319D31D7259E3132
:103C74008731E5279E319E3158260800F100240043
:103C840016157808023E8600870101080319552E8F
:103C94007108F0007808023E86008701010886005A
:103CA4008701700881002000EE01080021009112B4
:103CB4001112483023009F0090309D0026309E0052
:103CC40068309B009C012000EC01ED014030A00015
:103CD40020082100ED00E8019116080014302000AE
:103CE400A8007930A700A70B752EA80B752E0032FB
:103CF40032309F3181279E3128309F3181279E3178
:103D04000C309F3181279E3101309F3181279E31B4
:103D140006309F3181270800403021006D020318CE
:103D2400AB2E20006D08A03E8600023087000108FB
:103D340023009A000130F00070082000ED074030A5
:103D44006D020318ED010130F00070082100ED0749
:103D540008001112080023001908F0007008F1008F
:103D64002000911208307702031808007108F0004F
:103D74007708DB3E8600013087007008810001303F
:103D8400F0007008F707083077020318F7010130D4
:103D9400F0007008EB0708002000AC000230270296
:103DA4000318080010302C02031808002703031915
:103DB400DD2E8030DE2EC0302C04AA000030AB0093
:103DC4002A089F3181279E3107302000A9007D30C9
:103DD400A800A80BEB2EA90BEB2E08002000A600D0
:103DE4000730A5007D30A400A40BF62EA50BF62EFB
:103DF4002000A001A00A26089D31F8259E3120004C
:103E04002608A4000330A435FF3E031D052F2435E6
:103E1400A5002508A600A001A00A26089D31F825C2
:103E2400080022008C01FF3021008C0001302300A7
:103E34008C0022008D01013021008D0023008D01B2
:103E440024008D01183022008E00FB3021008E00EA
:103E5400220090010F3021009000240090012100E5
:103E6400951722009D0108002000AC012808AA0033
:103E74002708A9002C08290784002A0803182A0AFD
:103E840085001200031908002808AA002708A900C1
:103E94002C08290784002A0803182A0A8500000828
:103EA4009E31F0269F3101302000A9002908AC077B
:103EB400382F2000A10021006D0803195D2F111A6D
:103EC400682F2000210823009A007E2F1112200061
:103ED4002108A0006C08A03E86000230870020085C
:103EE40081000130A0002008EC0740306C02031868
:103EF400EC0101302100ED02210011160800200020
:103F0400A6000730A5007D30A400A40B872FA50BC5
:103F1400872F2000A00126089D31F8259F3120001D
:103F24002608A4000330A435FF3E031D952F243535
:103F3400A5002508A600F930A4000000A40B9F2FBB
:103F4400003200002000A00126089D31F825080059
:103F540003302000A3002308A0006730A1008330B1
:103F6400A2000030803103209F3103302000A300E1
:103F74002308A000A430A1008330A20000308031C7
:103F840003209F3104302000A3002308A000DF3069
:103F9400A1008430A2000030803103209F3187319A
:103FA400FE2708002000BC00BF013908A70038081C
:103FB400A6003D30BA003A08A8003708AA0036081F
:103FC400A9003F30BB003B08AB003C0894315F24A0
:103FD4009F31003A031DF12F20003F0808000130F3
:103FE4002000B6070030B73D3D08B8023E08B93B93
:0C3FF40038083904031DD72F3F080800CF
:020000040001F9
:04000E00E4C1FFDC6E
:00000001FF
